:020000040000FA
:020000003A299B
:080008008B138B1B0428B300CD
:10001000030EB40083010A08B5008A0183130408A3
:10002000B6008B181B2814281A08B2003014831647
:100030008C1283126B28311C3F283708073C031CA5
:100040002728381C861138188615B80C6D283708F3
:10005000083C031C3028B11C8611B11886156D2888
:100060003708093C031C38288316861583126D282F
:1000700037080B3C031C6D28B70131106E28B708F8
:10008000031D4528861968286D283708083C031C7D
:100090005128861DB8138619B81703196D28B80C96
:1000A0006D283708093C031C56286D28861D6828D2
:1000B00031196128B01483160610831206100B1232
:1000C00069283B083802031D68283111B7016E28E2
:1000D000B801B7016E288C126F28B70A8B1036084A
:1000E000840035088A00340E8300B30E330E0900F5
:1000F0008520B1197E2883161810802883161814BD
:10010000981C8028831299000800AA00A7000830D4
:10011000A800A9012718A90AA70CA80B8A28B111C1
:10012000291CB1152A0808000B1283160610861127
:100130008312061086115030A000A00B9D28B70135
:1001400083160614831231148B100B163118A6284F
:100150000800A2000830A300A4012218A40AA20CDF
:10016000A30BAD28B110241CB1140800BB0031153D
:100170003119B82808003808F03C031DC128311691
:10018000FE283808E03C031DC728B116FE283808B1
:10019000E13C031DCD283117FE28B11ADB28311BA5
:1001A000E62802308A0038080022311AF528FF3983
:1001B000031D7820FE2803308A0038080023311AF6
:1001C000F528FF39031D7820B112FE283808773C46
:1001D000031DFE28311AF028003078203113FE2844
:1001E0008030782031123113FE28FF390319FA28A4
:1001F000803878203112B1123113FE28831606148C
:100200008312B0100B16080032182129321E0C2957
:100210006E30782000307820B21EBA10B21ABA14AC
:10022000321F3A11321B3A15ED30B800A920942044
:10023000FA30B6203A08B800A9209420FA30B62047
:100240003529B21C25290330BA06321D3A1032195D
:100250003A14ED30B800A9209420FA30B6203A08BC
:10026000B800A9209420FA30B620301083168C16DE
:100270008312080083168101061486158312F83054
:100280008B0583161811FF309900831218179817E1
:1002900083168C16181798168312C0308B04181604
:1002A00007309F00831606148615011383129030C1
:1002B0008B040B100230BA00B701B001B101AA30B3
:0C02C000B620B018BB20301804216129C2
:10040000820700345E3400345A345834563457343A
:10041000613400345F345D345B345934083436342D
:1004200000340034533405340034023409340734C2
:1004300000340034003413340B340A340F340D34D8
:10044000003400341B3414341134103415340E3499
:100450000034003452341C34123418341734163437
:1004600000340034243423341A3419341F341D3436
:100470000034003400342B34213420341E3425342D
:10048000003400342C342234273428342D342634DC
:10049000003400343334343429342A342F342E34A5
:1004A0000034003400343134003430343534003416
:1004B00000340334043432343734003438340034F4
:1004C00000340034003400340034003400343C3450
:1004D00000340034393400343E34423400340034C3
:1004E00000343A3441343F344434453443340634E0
:1004F0006A3460346D3440344B346C344A34633481
:1005000000340034003400345C34003400340034EF
:10051000003400340034003400340034003400343B
:020520000034A5
:1006000082070034003400340034003400340034F5
:10061000003400340034003400340034003400343A
:10062000003400345434623400345534003400341F
:10063000003400340034003400340034003400341A
:10064000003400340034003400340034003400340A
:1006500000340034003400340034003400340034FA
:1006600000340034003400340034003400340034EA
:1006700000340034003400340034003400340034DA
:1006800000340034003400340034003400340034CA
:100690000034003400346B3400340034003400344F
:1006A00000340034003400340034003400340034AA
:1006B0000034003400345134003400340034003449
:1006C000003400340034003400340034003400348A
:1006D0000034003468340034483466340034003464
:1006E000003465343D34493400344F3450340034E0
:1006F000003400340034693400340034673400348A
:100700000034003400340034003400340034003449
:100710000034003400340034003400340034003439
:100720000034003400340034003400340034003429
:100730000034003400340034003400340034003419
:02074000003483
:00000001FF
